:1000000046288A0182000D340A34533444342D3496
:1000100043346134723464343E34003420344F3419
:10002000703465346E34003420345734723469349B
:10003000743465340034203443346C346F34733496
:100040006534003420342D342034613462346F340C
:100050007234743400348A0182070D3457282034F6
:100060005E285734EB285234F9284134FB285A349F
:10007000E4285334E0285534E22843341529583411
:100080003229543479203F344C2100348316043013
:1000900085000230860006309F0070308F000230ED
:1000A0009000831200309200AE01AF013722E220AF
:1000B0000519572803303E21A014B821E921A400D6
:1000C000A50125082B20003A0319742824060319DA
:1000D0006C28A50AA50A6128A50A25082B205E28F8
:1000E000E22022303E215728203002223F300222D7
:1000F00057285421A1000E303E21AE01AF019920B6
:100100000318080014303E21AD010730A7002D0868
:10011000A6202108AD072D08443A031D8728A70B08
:1001200087281B303E21C3200318080022303E21BF
:100130000800E02059303F222221D6200314003A43
:10014000031D0800D120A21403100800A800A21C5F
:10015000AD28FC303F22A21028083F220310AB0B31
:100160000800AC0B08003E223E22A214AE0A03197E
:10017000AF0A3E22FF3A0319B9283E22FF3A031D77
:10018000BD28D1200800A218C828FF30A620C32807
:10019000FD303F22D620A021D620A0210310E2204E
:1001A00008000030AB000230AC000800FA30E60076
:1001B0003E22FF3A031DDE28E60BD828FF3A08004E
:1001C00086110800861508005421A500FF303F2243
:1001D000A50BE6280800AC21E020E921203A031D08
:1001E000F7288B21031874283F22A021ED28E22054
:1001F00008002011FC282015AC2154216108A6001C
:100200006208A500E02005197028FF303F22201D5C
:10021000A0212019B321FF30A507031CA60726083B
:100220002504031D0329E2200800AC21E02054210D
:10023000403E3F2254216108AF006208AE002221F7
:10024000E22008002F08E1002E08E20047216008A4
:100250003F2261083F2262083F2200303F22953052
:100260003F220800AC215421A5008B21AD00E020E5
:100270002D083F22A50B3829E2200800DD005D088B
:100280000120003A031908000222DD0A3F29031069
:10029000E20DE10DE00D080054216008A021610885
:1002A000A0216208A0210800E001E101E201E921AA
:1002B000A4003030A402031C6C290A302402031865
:1002C0006C296E212408E207031C57290130E1073D
:1002D000031C5729E00A5729620808000310E20DA1
:1002E000E10DE00D6208B2006108B1006008B000E5
:1002F0000310E20DE10DE00D0310E20DE10DE00D44
:100300003208E20731080318310FE10730080318FB
:10031000300FE0070800B301972103180800B3006D
:10032000B30E972103180800330703100800E921D2
:1003300003180800BF3E031C073E0A3E03100800D6
:10034000B30020300222330EA62133080F39F63EC7
:100350000318073E3A3E022A0D3002220A300222DA
:1003600032304B220800E03E031C0030203E022ABF
:10037000B4011922033A0319E729033AF821E400EA
:100380000A3A0319B9296408083A0319D929340823
:10039000353E840064088000A01864080D3A0319F3
:1003A000E72964080222B40A3408273A0319E3292A
:1003B000B929B403B41BB829083002222030022224
:1003C00008300222B92908300222B403B929B40145
:1003D00008003408353E84000008B40A0D3A0319B9
:1003E000B4030D3AA4002F3C24080800B40308000D
:1003F0009F3E031C002AE63E0318203E5B3E080099
:10040000613E0800A400E501E5150A304B222D22CB
:1004100085102D2200000000000000000000A40C48
:10042000031C8510031885142D22E50B0E2A851454
:100430000800E501E515A401051D1C2A3222051D51
:10044000192A2D220310051D0314A40C000000001E
:10045000E50B212A2D22240808000A30E600E60BCD
:100460002F2A08000430E600E60B342A0800831621
:10047000C03094008312303094000800FF309300A5
:100480008316141C412A831213080800A02132305D
:100490004B2200300800E800E700E600E60B4E2A99
:0A04A000E70B4D2AE80B4C2A080078
:02400E00222F5F
:00000001FF
